:020000040800F2
:10000000005000207513000845130008491300082C
:1000100000000000000000000000000000000000E0
:100020000000000000000000000000006513000850
:1000300000000000000000006713000869130008BA
:10004000C5130008C5130008C5130008C513000830
:10005000C5130008C5130008C5130008C513000820
:1000600000000000C5130008C5130008C5130008F0
:10007000C5130008C5130008C5130008C513000800
:10008000C5130008C5130008C513000800000000D0
:10009000C5130008C5130008C5130008C5130008E0
:1000A000C5130008C5130008C5130008C5130008D0
:1000B000C5130008C5130008000000000000000080
:1000C00010B5064C2378002B07D1054B002B02D02E
:1000D000044800E000BF0123237010BD0C00002085
:1000E00000000000E4370008044B10B5002B03D0DB
:1000F0000349044800E000BF10BDC04600000000F6
:1001000010000020E4370008002243088B4274D31B
:1001100003098B425FD3030A8B4244D3030B8B4208
:1001200028D3030C8B420DD3FF22090212BA030C11
:100130008B4202D31212090265D0030B8B4219D3F2
:1001400000E0090AC30B8B4201D3CB03C01A524112
:10015000830B8B4201D38B03C01A5241430B8B425A
:1001600001D34B03C01A5241030B8B4201D30B0343
:10017000C01A5241C30A8B4201D3CB02C01A52416A
:10018000830A8B4201D38B02C01A5241430A8B422D
:1001900001D34B02C01A5241030A8B4201D30B0216
:1001A000C01A5241CDD2C3098B4201D3CB01C01A30
:1001B000524183098B4201D38B01C01A524143093A
:1001C0008B4201D34B01C01A524103098B4201D328
:1001D0000B01C01A5241C3088B4201D3CB00C01A95
:1001E000524183088B4201D38B00C01A524143080D
:1001F0008B4201D34B00C01A5241411A00D2014632
:10020000524110467047FFE701B5002000F0F0F8BA
:1002100002BDC0460029F7D076E7704703460B437E
:100220007FD4002243088B4274D303098B425FD3EF
:10023000030A8B4244D3030B8B4228D3030C8B421B
:100240000DD3FF22090212BA030C8B4202D3121201
:10025000090265D0030B8B4219D300E0090AC30BD6
:100260008B4201D3CB03C01A5241830B8B4201D383
:100270008B03C01A5241430B8B4201D34B03C01A6C
:100280005241030B8B4201D30B03C01A5241C30AE4
:100290008B4201D3CB02C01A5241830A8B4201D355
:1002A0008B02C01A5241430A8B4201D34B02C01A3F
:1002B0005241030A8B4201D30B02C01A5241CDD2E4
:1002C000C3098B4201D3CB01C01A524183098B422F
:1002D00001D38B01C01A524143098B4201D34B0118
:1002E000C01A524103098B4201D30B01C01A52417B
:1002F000C3088B4201D3CB00C01A524183088B4202
:1003000001D38B00C01A524143088B4201D34B00EA
:10031000C01A5241411A00D201465241104670475C
:100320005DE0CA0F00D04942031000D34042534061
:1003300000229C4603098B422DD3030A8B4212D321
:10034000FC22890112BA030A8B420CD38901921153
:100350008B4208D3890192118B4204D389013AD090
:10036000921100E08909C3098B4201D3CB01C01A65
:10037000524183098B4201D38B01C01A5241430978
:100380008B4201D34B01C01A524103098B4201D366
:100390000B01C01A5241C3088B4201D3CB00C01AD3
:1003A000524183088B4201D38B00C01A5241D9D2EB
:1003B00043088B4201D34B00C01A5241411A00D26C
:1003C0000146634652415B10104601D34042002B68
:1003D00000D54942704763465B1000D3404201B5E7
:1003E000002000F005F802BD0029F8D016E770479C
:1003F0007047C046844608006146FFE71FB500F01D
:10040000B9F9002801D40021C8421FBD10B500F081
:1004100045F94042013010BD10B500F0ABF900289D
:1004200001DB002010BD012010BDC04610B500F05A
:10043000A1F9002801DD002010BD012010BDC0463B
:1004400010B500F051F9002801DC002010BD01209A
:1004500010BDC04610B500F047F9002801DA0020B1
:1004600010BD012010BDC046002B11D1002A0FD1B4
:10047000002900D1002802D00021C943080007B498
:10048000024802A14018029003BDC04665FFFFFF6D
:1004900003B4684601B5029800F034F8019B9E460B
:1004A00002B00CBC7047C046F0B5CE469946030C6E
:1004B0009C46130447461B0C1D000E0061460404B5
:1004C000240C80B50700100C4B4365434143604347
:1004D0002C0CC01820188C46834203D980235B0261
:1004E0009846C444494679435643030C2D042D0CC9
:1004F0008919634400044019C918C0BCB946B04604
:10050000F0BDC046F0B557464E464546DE46E0B51E
:1005100004000D009246994683B08B4230D82DD00E
:100520004946504600F07CFB29000600200000F000
:1005300077FB331A9846203B34D49B4653465A46A1
:10054000934042461F00534693401E00AF423BD8A3
:10055000AF4200D179E05B46A41BBD41002B00DA1D
:1005600076E0002200230092019301235A46934033
:100570000193012342469340009329E08242CFD960
:1005800000220023009201930C9B002B01D01C60E1
:100590005D600098019903B0F0BCBB46B246A94625
:1005A000A046F0BD42469B4620239B1A5246DA40A5
:1005B000414613004A468A40170042461F435346AD
:1005C00093401E00AF42C3D9002200230092019342
:1005D0004346002BD8D0FB0772081A4346467B08D7
:1005E0000EE0AB4201D1A2420CD8A41A9D410120D9
:1005F00024196D410021013E24184D41002E06D0E2
:10060000AB42EED9013E24196D41002EF8D100987D
:1006100001995B4600196941002B24DB2B005A46E7
:100620004446D3402A00E2401C005B461500002BE4
:100630002ADB26009E40330026004746BE4032009B
:10064000801A9941009001919EE7A342BCD882E7AD
:100650004246202300219B1A002200910192012290
:10066000DA40019285E7424620239B1A2A0046463B
:100670009A402300F340444613432A00E2401C0002
:100680005B461500002BD4DA42462F0020232600BB
:1006900097409B1ADE403B003343CDE770B54200E4
:1006A00045024E024C00C30F6D0A0120120E760A5D
:1006B000240EC90FFF2A06D0FF2C03D0A24201D17D
:1006C000B54206D070BD002DFCD1FF2CFAD1002E12
:1006D000F8D18B4206D00120002AF3D12800431E16
:1006E0009841EFE70020EDE770B5420045024E0269
:1006F0004C00C30F6D0A120E760A240EC80FFF2A93
:100700001BD0FF2C0ED0002A1BD1002C01D1002EB3
:100710001CD0002D0CD083421CD00221581E084052
:10072000013870BD002E22D1002AF4D1002DF2D163
:100730000028F6D101204042F3E7002D17D1FF2C0D
:10074000F0D0002CE7D1002EE5D1E6E70020002D07
:10075000E7D0E2E7A24205DCEADBB54202D8E7D304
:100760000020DEE74342584140000138D9E702202B
:100770004042D6E770B5420045024E024C00C30F1E
:100780006D0A120E760A240EC80FFF2A0BD0FF2C1A
:100790000DD0002A1FD1002C16D1002E14D100201C
:1007A000002D10D009E0002D0CD1FF2C13D1002E0C
:1007B00008D1002A08D0834212D00221581E0840D6
:1007C000013800E0022070BD002DF4D10028FAD1DC
:1007D00001204042F7E7002CEDD1002EEBD1ECE7F1
:1007E000A24205DCF2DBB54202D8EFD30020EAE7F3
:1007F0004342584140000138E5E7C04643025B0AE6
:10080000F0B54F4646469946D646C30F4500984632
:10081000C0B54B460F1C2D0E00D1CBE0FF2D00D1F3
:10082000CFE08022DB00D2041A4300239146002649
:100830009A467F3D7C027B00640A1B0EFF0F002B53
:1008400000D1A9E0FF2B11D08022E400D204144390
:1008500042467F3B5B197A400020D2B25D1C0A2ED3
:1008600013DD3A000B2E47D047463FE02B00FF3305
:10087000002C1ED102221643424601357A40D2B2E4
:10088000FF350A2E00DDE4E00220022E1CDC013ED2
:10089000012E42D802283DD0012866D10020002137
:1008A000C0050843D2071043E0BCBA46B146A8468B
:1008B000F0BD03221643424601357A40D2B2FF35DD
:1008C0000A2E00DDE4E003200121B140A626F60057
:1008D00031420AD19026B600314216D1B93EFF3ED0
:1008E0000E421AD0A146824600E0170053463A0055
:1008F000022B0FD04C4650460328CDD18021C9038E
:1009000021434902FF20490ACAE780210022FF2033
:10091000C903C5E7FF200021C2E7200C4946240493
:10092000240C27000E0C0904090C74434F43464362
:100930004843390C001909188C4203D98020400221
:10094000844666443F0408043F0CC0198401671EB6
:10095000BC41090C800E8919044389010C4309012B
:1009600071D5012361081C400C432B007F33002B01
:1009700051DD610704D00F212140042900D0043447
:10098000210103D5434B1C402B008033FE2BC1DCDF
:10099000A101490AD8B283E7002C2CD10123424699
:1009A0001E432B007A400120D2B25D1C0A2E00DDCE
:1009B00057E76AE7002B10D10123042600259A4649
:1009C00038E7002B04D102230826FF259A4631E799
:1009D00003230C26FF259A462CE7484600F002F92F
:1009E0004A46431F76259A4000236D4291460026D1
:1009F0009A462D1A1EE7200000F0F4F84246431FE5
:100A00009C402B1A763B7A400020D2B25D1C0A2E05
:100A100000DD26E739E70121CB1A1B2B00DD3DE77E
:100A20009E352100AC40D940631E9C4121434B07B9
:100A300004D00F230B40042B00D004314B0104D50C
:100A4000012000212CE71D008FE789010020490AC1
:100A500026E702230F2E0CD180214B46C9030B42FF
:100A60000DD00C420BD1214349023A00FF20490A24
:100A700016E70B2E00D0F7E6A1469A4636E780210E
:100A80004B46C903194349024246FF20490A07E77A
:100A90000323DFE7FFFFFFF741024200C30F490ACC
:100AA0000020120E7E2A03DD9D2A02DD094A9818D5
:100AB0007047802000040143952A07DC9620821AA3
:100AC000D1404842002BF3D10800F1E7963A91401B
:100AD000F7E7C046FFFFFF7F0200F0B54B000D03B4
:100AE000400F5B0DCC0F6D0A3A490543581CD700E7
:100AF00008420AD038495918FE2916DDFF20002285
:100B0000C0051043E4072043F0BD002B06D13D4350
:100B100026D005229201520AD8B2F1E72F43EDD038
:100B20008022D203FF202A43EAE700291BDD92013D
:100B3000501E8241ED007F0F2A433A43530747D0AE
:100B40000F231340042B00D004328023DB04134016
:100B50003ED0481CFE29D1D09201520AC0B2CFE744
:100B600000200022CCE70A0017322FDB8026360453
:100B70002E431E256D1A1F2D11DD02225242521ADC
:100B80003100D140202D04D0144A944663449E4045
:100B900037433A00531E9A410A430021CEE7104AD8
:100BA00038009446634498403A00411E88419E4074
:100BB000EA403043024300215307C1D18021130092
:100BC000C90401200B400A42C6D1A3E70023A0E7D5
:100BD0000B009FE7FE07000080FCFFFFA2FCFFFF69
:100BE00082FCFFFF1C2101231B04984201D3000C4F
:100BF00010391B0A984201D3000A08391B09984290
:100C000001D30009043902A2105C40187047C046A5
:100C100004030202010101010000000000000000C5
:100C200010B5002903D1FFF7DDFF203002E00800F6
:100C3000FFF7D8FF10BDC046F0B589B014220021DF
:100C400003A802F098FD1A4BDA6A01252A43DA62FA
:100C5000DA6A2A400192019AD96A04221143D962C0
:100C6000DB6A1A400292029B81242401A027FF051F
:100C700000222100380000F01DFF0E4E002210213E
:100C8000300000F017FF03940495002405940694A7
:100C900003A9380000F016FE102303930495059471
:100CA000069403A9300000F00DFE09B0F0BDC04667
:100CB000001002400008005000B593B0342200211B
:100CC00005A802F058FD14220021684602F053FDE9
:100CD00017490A68174B1A4080231B0113430B6006
:100CE00002230593012208920F3209920E930023EA
:100CF0000F938023DB0210938023DB03119305A85D
:100D000000F038FF00280FD10F2300930C3B019314
:100D100000230293039304930121684601F0ECF948
:100D2000002803D113B000BD72B6FEE772B6FEE72D
:100D300000700040FFE7FFFF30B583B00E4CA37892
:100D4000627821780D48E578009502F085FA6168AF
:100D50000B4802F081FA21890A4802F07DFA618984
:100D6000094802F079FAA189084802F075FA64206E
:100D700000F076FB03B030BD3801002000380008D9
:100D800010380008203800083038000840380008C3
:100D900010B5642000F064FB72B600F0A5FB10BD36
:100DA0000E4B1B78013BDBB2FD2B11D80B4B5B6864
:100DB000013B03330ED8094B1B89013B9BB2084A08
:100DC000934209D8054B9889431E9841C0B200E070
:100DD000002070470020FCE70020FAE738010020DF
:100DE000FDFF0000F0B5DE4657464E464546E0B5ED
:100DF00083B000F00FFB02F03DFAFFF75DFFFFF755
:100E00001BFF00F03FFAFA24A400200000F028FBAA
:100E100002F0A6FCD24802F01FFA200000F020FBEE
:100E20008021A02000220901C00500F043FECD4B27
:100E300000221A701F00CC4B0193CC4B984642E025
:100E4000019802F009FA802002224146C00002F017
:100E500095FA43461988C64802F0FEF9C549A02014
:100E60001022C00002F08AFAFFF766FF43461A8894
:100E7000531E9BB2C0498B420AD8C04B9A4200D045
:100E8000BEE0FFF78DFF012800D18EE0BC4908E0ED
:100E9000B649BC4B0B8080200222C00002F04AFA07
:100EA000B749B94C2160B94802F0D6F9FA20C00020
:100EB00000F0D6FA2368B24A934200D1A2E0AF4ACA
:100EC000934200D1AAE0FA20800000F0C9FA3B78F2
:100ED000002BB5D0012BF6D1A24B5B78022B00D1B1
:100EE00005E100D9A0E0002B00D1B6E0A84802F04F
:100EF000B3F9A04CC02010222100C00002F03EFA3D
:100F0000FFF71AFFA025ED001021280002F04EFA8D
:100F100010222100280002F00DFA9E499E4802F09E
:100F200069FA2389002B3CD000249C4D9C4B9946A8
:100F3000904E9C4BE01800020122290002F09EFA1C
:100F400029782200484602F087F90134A4B2338997
:100F5000A342EED8002B24D00024934B9B468F4B0A
:100F60009946844B9A462100584602F075F980262E
:100F7000760032000021484602F0FDFBA5192D0243
:100F800032004946280002F0FBFA884BE81832008C
:100F9000494602F04CFA0134A4B253461B89A342DD
:100FA000E1D8704B02225A708DE7814B71490A6873
:100FB0001A60BF301022C00002F0E0F9FFF7BCFE5B
:100FC000FFF7EEFE012801D06D496AE7694B1A6808
:100FD000784B1A60D1B20A2359431202120E8A18B2
:100FE00073490878434389785B18D81700219342E6
:100FF00041414942704B1940604B9C46614450E767
:101000005F494EE7644802F061F9012800D05AE7D1
:101010006A4802F021F9FFF7BBFE54E7514B012269
:101020001A7000225A704EE7032B00D04BE7644839
:1010300002F012F94F49E0201022C00002F09EF9A0
:10104000FFF77AFEFFF7ACFE012800D1CCE05D4847
:1010500002F002F9FFF79CFE35E75B4802F0FCF86E
:10106000444CA02010222100C00002F087F9FFF7B5
:1010700063FEE025ED001021280002F097F9102210
:101080002100280002F056F9032002F0E5FA0420BE
:1010900002F0E2FA2389002B25D000244B4B9B461B
:1010A0003E4B9946334B9A462100584602F0D4F8FD
:1010B0008026760032000021484602F05CFB394B66
:1010C000E5182D0232004946280002F0D7F9404BBE
:1010D000E8183200494602F089FA0134A4B25346B6
:1010E0001B89A342E0D81F4B01225A70EBE6394816
:1010F00002F0B2F81F4CA02010222100C00002F024
:101100003DF9FFF719FE6168234802F0B7F80100C6
:10111000314D2880314802F09FF8A2892B889A42ED
:1011200006D02F4802F098F80E4B03225A70CAE6F8
:101130002C4802F091F80D49124B0B8080200222BE
:10114000C00002F0F7F8144802F0C0F8012800D0FF
:10115000B9E61A4802F080F8FFF71AFEB3E6C04677
:101160004C380008280000205C3800082C000020C3
:101170006C38000838010020FDFF0000BBBB0000F8
:10118000AAAA0000AAAAFFFF3000002080380008A9
:10119000BC3800087F030000004000083400002035
:1011A000CC38000840000800D43800080040FF0791
:1011B0004C01002048010020EFEEFFFF8C380008B2
:1011C000243900084C39000898380008A83800086D
:1011D00000C002F8E438000850010020F43800088C
:1011E0001439000804390008A025ED00102128005A
:1011F00002F0DCF81B4C10222100280002F09AF8C3
:1012000019491A4802F0F6F82389002B26D0002449
:10121000174B9B46174B9946124B9A46210058464E
:1012200002F01AF88026760032000021484602F0CB
:10123000A2FAC0239B00E5182D023200494628007F
:1012400002F09EF90C4BE8183200494602F0EFF824
:101250000134A4B253461B89A342DFD8074B0222B4
:101260005A7030E6380100207F030000004000087B
:1012700038390008340000200040FD072800002015
:1012800072B6FEE710B51048104B036082235B0076
:10129000436000238360C36002220261013A42611D
:1012A000802292008261F93AFF3AC261036243628E
:1012B00083620733C36201F01FF9002800D110BD1B
:1012C000FFF7DEFFFBE7C04654010020003001407D
:1012D00010B586B004001422002101A802F04BFAD8
:1012E0000F4B22689A4201D006B010BD0D4B596BCE
:1012F000802252010A435A63D96A01221143D962FA
:10130000DB6A1A400092009BE0230193DE3B0293CC
:1013100001330493A02001A9C00500F0D3FAE3E74C
:101320000030014000100240054B5A6B01210A4376
:101330005A63996B802252050A439A637047C046EC
:1013400000100240FEE7000070B5054DFA24A4002D
:10135000280001F081FF200000F082F8F8E7C04685
:10136000643900087047704710B500F067F810BD89
:10137000704700000D488546FFF7FAFF0C480D49FD
:101380000D4A002302E0D458C4500433C4188C42E0
:10139000F9D30A4A0A4C002301E013600432A24246
:1013A000FBD302F0F1F9FFF71DFDFEE7005000202E
:1013B000000000200C000020203B00080C00002052
:1013C00080060020FEE7000070B504000E4D0F4BB4
:1013D0001978FA208000FEF797FE01002868FEF7D2
:1013E00093FE00F08FF800280BD10130032C09D8B0
:1013F00000222100404200F045F8054B1C6000200F
:1014000000E0012070BDC046000000200400002064
:101410000800002010B5084A136840210B431360F0
:101420000320FFF7D1FF041E02D00124200010BDCD
:10143000FFF77AFFFAE7C04600200240034A11682E
:10144000034B1B785B1813607047C046AC0100204B
:1014500004000020014B18687047C046AC01002012
:1014600070B50400FFF7F6FF0500631C02D0044BC3
:101470001B78E418FFF7EEFF401BA042FAD370BDC3
:101480000400002070B5002814DB8408A400144B6D
:101490009C466444C026B600A55903220240D200EF
:1014A000FF2318009040854389010B4093402B4354
:1014B000A35170BD0F230340083B9B089B00094AC2
:1014C00094466344DC6903221040C000FC321500DE
:1014D0008540AC4389010A4082402243DA61E8E753
:1014E00000E100E000ED00E0BFF34F8F034B044A42
:1014F000DA60BFF34F8FC046FDE7C04600ED00E065
:101500000400FA05013880235B0498420FD2094A8F
:1015100050600948036A1B021B0AC02109060B43DD
:10152000036200239360073313600020704701209B
:10153000FCE7C04610E000E000ED00E02B4B9969AD
:10154000802252000B001340114206D0284A5369F2
:1015500002210B43536180235B00244A9269920568
:1015600007D523494A69012002434A61802292003B
:1015700013431E4A9269520507D51D494A6908203E
:1015800002434A618022D2001343184A926912052D
:1015900007D517494A69042002434A618022120193
:1015A0001343124A9269920407D511494A691020DF
:1015B00002434A618022920113430C4A92699203CA
:1015C00005D50B48426920210A4342610B43074A73
:1015D0009269D20307D506494A69402002434A610D
:1015E000802252021343014A936170470020024057
:1015F000B0010020124B5B68DB070CD5EFF31082C3
:1016000072B60F4B0F49D9600F49D96082F3108829
:101610005B68DB0712D40A4B5B6800209B070CD584
:10162000EFF3108272B6064B084919610849196137
:1016300082F3108858688007C00F70470120FCE7CC
:1016400000200240EFCDAB8905040302BFAE9D8CA4
:1016500016151413054B5A6802210A435A605A683A
:1016600001390A435A6000207047C04600200240FA
:10167000F8B50400FFF7EEFE07001D4E0125B36923
:101680001D420AD0631CFAD0002C2ED0FFF7E2FED8
:10169000C01BA042F3D9032026E0154B9B699B0792
:1016A00002D5134B02229A61114B9B69DB0518D4BA
:1016B0000F4B9B699B0514D40D4B9B695B0510D4A4
:1016C0000B4B9B691B050CD4094B9B699B0408D4ED
:1016D000074B9B699B0304D4054B9B690020DB03EC
:1016E00002D5FFF72BFF0120F8BD0320FCE7C04621
:1016F0000020024070B50C0015000D4B1B7C012B27
:1017000013D00B4B01221A740A48FFF7B1FF0028CF
:1017100003D0074B00221A7470BD054B00225A619A
:1017200025600448FFF7A4FFF3E70220F4E7C04672
:10173000B001002050C30000094B5B680020DB07AC
:101740000CD5EFF3108272B6054B0649D9600649F5
:10175000D96082F310885B68013018407047C0463A
:1017600000200240EFCDAB8905040302034A536811
:1017700001210B43536000207047C0460020024007
:1017800010B504000648FFF773FF002800D010BD15
:10179000044B00225A6122600148FFF769FFF6E717
:1017A00050C30000B001002070B506000D00140009
:1017B000124B1B7C012B1FD0104B01221A741048B6
:1017C000FFF756FF002810D10C4B00225A61022E61
:1017D00007D0012E0DD00120002E06D1E4B22C70CE
:1017E00000E02C600648FFF743FF044B00221A7408
:1017F00070BDA4B22C80F5E70220F9E7B00100200B
:1018000050C3000010B5084B00215961074B5C68BC
:101810008022920022435A605A68082422435A6068
:101820007F239843016010BDB001002000200240DA
:10183000F8B5CE46474680B5060089461D4B1B7C51
:10184000012B35D01B4B01221A741B48FFF710FFE8
:10185000002826D101235B424A4613607468B368AE
:10186000DB011B199C421CD2134B9846134D0827D1
:101870002000FFF7C7FF4046FFF7FAFE6B68BB4347
:101880006B606B680E4A13406B60002807D1803490
:10189000B368DB0172689B18A342E9D801E04B46AC
:1018A0001C60044B00221A74C0BCB946B046F8BD97
:1018B0000220F9E7B001002050C3000000200240E0
:1018C000FFFDFFFFF0B5DE4657464E464546E0B504
:1018D00083B00E68002E00D1D4E000220023032440
:1018E000C025AD02AB466B4DAA466B4D45196F1E28
:1018F000BD410535019543E0866827009740BE430A
:10190000B446CE68964067463E4386604668AE431E
:101910004D682D0901273D409D40354345603BE022
:1019200000266746BE4047463E43AE605B4DAD680D
:10193000009EF6434F68FF0200D597E03540574FB1
:10194000BD60FD684F68BF0200D592E03540534F3F
:10195000FD607D684F68BF0300D58DE035404F4F77
:101960007D603D684F68FF0300D588E035404B4EF1
:10197000356001330E6802323500DD4000D181E070
:1019800001259D4037002F4000972E42F1D04E6830
:101990002640013E012EAFD94D682540032D24D0AD
:1019A000C66825009540AE438D6895403543C560B7
:1019B0004D682540022D18D1DD08AD00A9468144AF
:1019C0004D462E6AB04607261E40B6000F27B74088
:1019D000BC4647466546AF43B8460D692F00B74041
:1019E0003E0045462E434D462E6206682500954032
:1019F000AE434D6825409540354305604D685E46D1
:101A00003542B6D055466D6B012635435646756353
:101A10009D08AD00224EB4466544AE68B04626002F
:101A20001E40B600B4460F266746BE404746B74341
:101A3000B846A026F605B04200D171E7194EB1466E
:101A40000126484500D16CE7174EB0420AD0174E28
:101A5000B1462600484500D163E7154EB04203D099
:101A6000019E5EE702265CE704265AE7009F3D439D
:101A700065E7009F3D436AE7009F3D436FE7009E97
:101A8000354374E703B0F0BCBB46B246A946A04656
:101A9000F0BDC0460010024000E4FFAF000401406A
:101AA000000001400004005000080050000C0050ED
:101AB00000100050002A01D0816170478162FCE76C
:101AC00010B5264BDA680C231340082B43D00C2B9F
:101AD00014D0042B08D0214B5B681B045B0F01332F
:101AE00080200002984008E01C4B1868C006C01710
:101AF0001B4B18401B4B9C46604410BD1A49930277
:101B00001B0FC85C1202940F0134144BDB68DB031B
:101B100009D5164A00230021FEF7C6FC2200002347
:101B2000FEF7A2FCE9E70D4B1B68DB0609D5104A5E
:101B300000230021FEF7B8FC22000023FEF794FCEE
:101B4000DBE7084A00230021FEF7AEFC2200002359
:101B5000FEF78AFCD1E70548CFE7C04600100240F7
:101B600000E548FF0024F4008839000800127A00DC
:101B700000093D00F0B5D6464F464646C0B582B096
:101B8000041E00D199E2C24BDA680C251540DE68CC
:101B900080235B021E400368DB073CD5082D32D052
:101BA0000C2D2ED063688022520293425ED0A02278
:101BB000D202934261D0B64B1A68B6490A401A6005
:101BC0001A68802149020A400192019A1A68B249B2
:101BD0000A401A606368002B5BD0FFF73BFC0700EC
:101BE000AB4B994680239B0298464B461B68424666
:101BF000134210D1FFF72EFCC01B6428F5D9032037
:101C00005CE2002ECED0A24B1B689B0303D5636819
:101C1000002B00D158E223689B0775D5E3689A062C
:101C200005D59B48026820210A4302608B43042D9E
:101C300045D00C2D41D0002B00D1BCE094490A685E
:101C40000920824313430B60FFF704FC0600904B0E
:101C50009846042743461B681F4200D0A2E0FFF7C6
:101C6000F9FB801B0228F5D9032027E2884A116876
:101C700080235B020B431360ACE7854B196880221D
:101C8000D2020A431A601968802252020A431A607B
:101C9000A0E7FFF7DFFB07007D4B994680239B02FF
:101CA00098464B461B6842461342B4D0FFF7D2FB1E
:101CB000C01B6428F5D9032000E2002EBBD1744A72
:101CC0001268520702D5002B00D1FFE1704E7168F7
:101CD00022691202714801400A4372603268092188
:101CE0008A4313433360FFF7EBFEF3686C496D4A98
:101CF0001B061B0FD35CD84008606B4B1868FFF7BE
:101D000063FB002800D0D9E12368DB062CD5002D29
:101D100067D15F4B1B689B0503D5A369002B00D1DE
:101D2000D6E15B4B5A6861490A40216A0A435A600E
:101D30005968E26912060902090A0A435A60DA6818
:101D40005748216A490B013180231B028B405549BA
:101D50001206120F8A5CD3400360534B1868FFF7DA
:101D600033FB002800D0A9E123681B0700D4A1E0C1
:101D70006369002B76D0464A136D01210B4313652E
:101D8000FFF768FB0600424B9846022743461B6D4F
:101D90001F4200D08EE0FFF75DFB801B0228F5D9C3
:101DA00003208BE13A494A6823691B023B48024001
:101DB00013434B60A8E7364A136801218B43136035
:101DC000FFF748FB0600324B9846042743461B6842
:101DD0001F4299D0FFF73EFB801B0228F6D9032053
:101DE0006CE1A369002B26D0294A116880235B008F
:101DF0000B431360FFF72EFB0600254B9846802708
:101E0000BF0043461B683B4206D1FFF723FB801B04
:101E10000228F6D9032051E11D494B68234A13409B
:101E2000226A13434B604A68E3691B061202120AD6
:101E300013434B6098E7164A13681D490B40136023
:101E4000FFF708FB0600124B98468027BF00434669
:101E50001B683B4288D0FFF7FDFA801B0228F6D9A9
:101E600003202BE10A4A136D01218B431365FFF711
:101E7000F1FA0600064B9846022743461B6D1F42A7
:101E800018D0FFF7E7FA801B0228F6D9032015E1E6
:101E900000100240FFFFFEFFFFFFFBFFFFE0FFFF20
:101EA000000000207839000808000020FF1FFFFF15
:101EB000FFFEFFFF23685B0700D488E0864B9B6B27
:101EC00000229246DB0007D4834A916B80235B0596
:101ED0000B43936301239A46804B1B68DB0510D5A7
:101EE000A36880225200934223D0002B3ED17A4B2C
:101EF0001A6D7B490A401A651A6D7A490A401A65BB
:101F00001DE0764A116880235B000B431360FFF7E6
:101F1000A1FA0600714B984680277F0043461B6854
:101F20003B42DDD1FFF796FA801B6428F6D90320E7
:101F3000C4E0694A116D80235B000B431365A368FD
:101F4000002B2DD0FFF786FA0600634B98468027BA
:101F5000BF00654B994643461B6D3B4234D1FFF7AA
:101F600079FA801B4845F6D90320A7E0A022D200C9
:101F7000934209D0584B1A6D59490A401A651A6D97
:101F800058490A401A65DAE7534B196D013AFF3A8E
:101F90000A431A65196D802252000A431A65CEE77A
:101FA000FFF758FA06004C4B98468027BF004E4B6F
:101FB000994643461B6D3B4206D0FFF74BFA801B08
:101FC0004845F6D9032079E05346012B1CD0636ABB
:101FD0000020002B72D00C2D55D0022B1AD03E4A77
:101FE000136842490B401360FFF734FA04003A4E7D
:101FF0008025AD0433682B4243D0FFF72BFA001B3A
:102000000228F7D9032059E0334A936B38490B4033
:102010009363DCE7304A136834490B401360FFF7E1
:1020200019FA05002C4F8026B6043B68334206D0CF
:10203000FFF710FA401B0228F7D903203EE0264A9A
:10204000D168A36AE06A03432A4801400B43216B2D
:102050000B43D360116880235B040B431360FFF7CD
:10206000F9F904001C4E8025AD0433682B4206D1DB
:10207000FFF7F0F9001B0228F7D903201EE000202B
:102080001CE000201AE0012B24D0134BDB688022D7
:1020900052021A40A16A01208A420FD1F022920313
:1020A0001A40E16A8A4209D1C02212041340226B0D
:1020B0009B1A5A1E9341D8B200E0012002B0E0BC46
:1020C000BA46B146A846F0BD0120F7E70120F5E782
:1020D0000120F3E70120F1E700100240007000400A
:1020E000FFFEFFFFFFFBFFFF88130000FFFFFFFE67
:1020F000FFFFFFEFFFFF02FFF8B5CE46474680B572
:1021000004000D00002800D1E2E0734B1A6801239F
:1021100013408B421AD323689B0706D56F4AD368B6
:10212000F0218B43A1680B43D3602368DB0700D405
:102130008AE06268022A23D0032A46D0012A4AD0C4
:10214000664B1B689B0520D40120A7E0624A1368F8
:1021500001218B432B431360FFF77CF906005E4B94
:10216000984601275E4B994643461B683B40AB426D
:10217000D1D0FFF76FF9801B4845F5D903208DE0DA
:10218000564B1B689B0300D4A4E05449CB68032042
:1021900083431343CB60FFF75DF906006368022BAE
:1021A0001FD0032B2ED0012B3DD04C4B98460C2733
:1021B0004B4B99464346DB681F4245D0FFF74AF92F
:1021C000801B4845F6D9032068E0444B1B689B01FF
:1021D000DBD4012062E0414B1B685B07D5D40120B2
:1021E0005CE03E4B98460C273D4B99464346DB68E6
:1021F0003B40082B28D0FFF72DF9801B4845F5D927
:1022000003204BE0354B98460C27354B9946434607
:10221000DB683B400C2B17D0FFF71CF9801B4845AF
:10222000F5D903203AE02D4B98460C272C4B9946C4
:102230004346DB683B40042B06D0FFF70BF9801BBD
:102240004845F5D9032029E0234B1A6801231340A0
:10225000AB4227D823685B0706D5204AD3682149BB
:102260000B40E1680B43D36023681B0707D51B496C
:10227000CA682369DB001C4802401343CB60FFF7A8
:102280001FFC164BDB681949194A1B061B0FD35C50
:10229000D8400860174B1868FFF796F8C0BCB946DD
:1022A000B046F8BD0C4A136801218B431360FFF759
:1022B000D1F80500084F0126094B98463B681E429D
:1022C000C8D0FFF7C7F8401B4045F7D90320E5E722
:1022D0000120E3E70120E1E7002002400010024076
:1022E00088130000FFF8FFFFFFC7FFFF000000207A
:1022F0007839000808000020F0B5D6464F4646461B
:10230000C0B582B081460D0017001E00FFF7A2F88D
:102310000A9B9B191B1A9846FFF79CF88246304B84
:102320001B685B011B0D4246534301934B461B68E0
:102330009C682C40641B62425441BC4249D0721CD0
:10234000F6D0FFF787F85346C01A404507D2019BE5
:10235000002B00D19846019B013B0193E6E74B46D9
:102360001A685368E0218B43536082235B004A461E
:1023700052689A420ED080239B014A46926A9A4242
:1023800019D0512301224946CA54013B0022CA54A4
:1023900003201FE04B469B6880221202934203D029
:1023A0008022D2009342E6D14B461A68136840213E
:1023B0008B431360DFE74B461A68136809490B40EB
:1023C00013604B461A68116880239B010B4313600E
:1023D000D7E7002002B0E0BCBA46B146A846F0BD3F
:1023E00000000020FFDFFFFF70B584B004000D0087
:1023F0001600184B18681849FDF786FE02004301C5
:102400001B1A98008018C000039082235B0061684B
:10241000802299420BD0039B002B17D0039B013BDA
:10242000039323689B681A42F5D100200FE00096C1
:102430002B00002280212000FFF75EFF002806D03D
:10244000636D202213436365032000E0002004B085
:1024500070BDC0460000002000366E0130B583B06C
:1024600004000B00822040006568854209D000927C
:10247000002201212000FFF73FFF002835D103B0E3
:1024800030BDA16880200002814203D08020C000BE
:1024900081420ED1206801684025A9430160822154
:1024A000490060688842E2D18021C900A068884262
:1024B0000DD00092002280212000FFF71DFF002890
:1024C000DDD0636D2022134363650320D7E70092BC
:1024D000002201212000FFF70FFF0028CFD0636DFD
:1024E0002022134363650320C9E7636D2022134351
:1024F00063650320C3E7000070B5041E5ED0436A25
:10250000002B07D10533FF3342689A4205D00023E0
:10251000C36102E00023036143610023A3625133DE
:10252000E35C002B43D051220225A55421680B689F
:10253000402083430B6021686368C4300340A06877
:102540008426360230400343E0688026360130405E
:1025500003432069284003430120656905402B435C
:10256000A5698026B60035402B43E569C93EFF3E8C
:1025700035402B43256A483635402B43A56A8026D3
:10258000B60135402B430B602568618B04230B405B
:10259000616A102631400B436B602168CB69084D9E
:1025A0002B40CB6100236365A054002070BD5033E5
:1025B0000022E2542000FEF78BFEB4E70120F5E78D
:1025C000FFF7FFFFF0B5C64600B584B004000191E7
:1025D00017001D005023C35C012B00D1D4E0502311
:1025E0000122C254FEF736FF06005123E35CDAB243
:1025F0009046012B00D0BDE00199002900D1BBE03D
:10260000002F00D1B8E050330322E2540023636569
:102610002163A786E786A363A387E38763642364B4
:1026200080231B02A2689A4222D0226813685B06AC
:1026300003D4136840210B43136080231B01E2681D
:102640009A4221D06368002B01D0012F0AD1236860
:10265000226B12781A73236B01332363E38E013BE1
:102660009BB2E386E38E9BB2002B67D002274EE03D
:102670002268136840218B4313602268116880230D
:10268000DB010B431360D0E76368002B01D0012FFF
:102690000AD12368226B1288DA60236B023323632A
:1026A000E38E013B9BB2E386E38E9BB2002B45D0C9
:1026B00002270AE0FEF7CEFE801BA84214D36B1C53
:1026C00014D1E38E9BB2002B38D023689A6817424E
:1026D000F0D0226B1288DA60236B02332363E38E1F
:1026E000013B9BB2E386ECE7002DEAD151230122A6
:1026F000E2544E3B98463FE0FEF7ACFE801BA842FA
:1027000014D36B1C14D1E38E9BB2002B16D023681C
:102710009A681742F0D0226B12781A73236B013338
:102720002363E18E013989B2E186ECE7002DEAD11D
:1027300051230122E2544E3B98461DE0320029000D
:102740002000FFF751FE002801D020236365A36815
:10275000002B06D103932368DA6803929B680393E6
:10276000039B636D002B07D151330122E2540023F8
:10277000984601E00223984650230022E254404646
:1027800004B080BCB846F0BD02239846F7E7F0B528
:10279000D6464F4680B585B00400009101921F00D7
:1027A0000C9D5023C35C012B00D122E15023012258
:1027B000C254FEF74FFE06005123E35CD9B26268B3
:1027C000012B0CD082235B0002209A4200D000E152
:1027D000A368002B00D0FBE0042900D0F9E0009BA7
:1027E000002B00D1FDE0019B002B00D1FBE0002F6E
:1027F00000D1FAE05123E35C042B02D051230522DF
:10280000E25400236365019AA263E787A787009AD1
:102810002263E786A7862364636423681A685206E6
:1028200003D41A6840210A431A6080231B01E2681E
:102830009A4215D06368002B01D0012F0AD123687A
:10284000226B12781A73236B01332363E38E013BEF
:102850009BB2E38601239A4601339946012773E030
:102860006368002B01D0012F0AD12368226B1288E4
:10287000DA60236B02332363E38E013B9BB2E38672
:1028800001239A460133994601271BE02268936889
:10289000390019401F420ED0E38F9BB2002B0AD0A3
:1028A000D268A36B1A80A36B0233A363E38F013B4F
:1028B0009BB2E3878A46FEF7CDFD801BA84201D379
:1028C0006B1C20D1E38E9BB2002B03D1E38F9BB214
:1028D000002B61D023689A6849461142D6D0E28E17
:1028E00092B2002AD2D05246012ACFD1226B12884E
:1028F000DA60236B02332363E38E013B9BB2E386F2
:1029000000239A46C2E751230122E254032060E0EB
:1029100022689368390019401F420ED0E38F9BB2A2
:10292000002B0AD0D268A36B1A70A36B0133A36388
:10293000E38F013B9BB2E3878A46FEF78BFD801B4A
:10294000A84222D36B1C22D1E38E9BB2002B03D171
:10295000E38F9BB2002B1FD023689A68494611422F
:10296000D6D0E28E92B2002AD2D05246012ACFD1DE
:10297000226B12781A73236B01332363E38E013BBE
:102980009BB2E38600239A46C2E7002DDCD1512397
:102990000122E25403201CE0320029002000FFF74E
:1029A00023FD002810D1A368002B06D103932368D0
:1029B000DA6803929B680393039B636D002B16D127
:1029C00051330122E25404E020236365012000E03A
:1029D000022050230022E25405B0C0BCBA46B146E2
:1029E000F0BD0120F5E70120F3E70120F1E7012028
:1029F000EFE70220F0E70000F0B5CE4600B584B066
:102A00000400039116001D005123C35CDFB2012BAB
:102A100000D0ABE00433FF3342689A4244D05023E5
:102A2000E35C012B00D1AAE050230122E254FEF71F
:102A300011FD81460399002900D198E0002E00D1B4
:102A400095E051230422E25400236365A163A68725
:102A5000E6872363A386E3862364636480231B02E3
:102A6000A2689A422DD0226813685B0603D41368CB
:102A700040210B431360E368002B2DD0E38F9BB202
:102A80000126002B5CD14A4629002000FFF7E6FC16
:102A9000002801D020236365636D002B67D151337B
:102AA0000122E254002762E08368002BB7D1513342
:102AB0000422C254009533000A00FFF768FE0700A5
:102AC00058E02268136840218B4313602268136822
:102AD0002C490B401360C6E7E38F9BB2002BD2D08A
:102AE00001260BE0FEF7B6FC4B46C01AA84214D3F1
:102AF0006B1C14D1E38F9BB2002BC4D023689A685F
:102B00001642EFD0A26B1B7B1370A36B0133A36340
:102B1000E38F013B9BB2E387ECE7002DEAD1512321
:102B20000122E254032722E0FEF794FC4B46C01A30
:102B3000A84214D36B1C14D1E38F9BB2002BA2D0FC
:102B400023689A681642EFD0DA68A36B1A80A36BE9
:102B50000233A363E28F013A92B2E287ECE7002DE1
:102B6000EAD151230122E254032700E00227502337
:102B70000022E254380004B080BCB946F0BD022700
:102B8000F8E7C046FFBFFFFF0369C268934204D85D
:102B900081685B18013B981A7047013B981AFBE764
:102BA000F8B5CE46474680B504000E001700C5684C
:102BB000836899465B1B9846934209D9406840193F
:102BC00000F006FEED19E560C0BCB946B046F8BDA0
:102BD000406840191A0000F0FBFDED194B46ED1A54
:102BE0006068310041442A0000F0F2FDEBE7F8B5DF
:102BF000CE46474680B5060088461700C5680023C4
:102C0000994617E0B2689B18013B5B1B17E07068A0
:102C100040192200414600F0DBFDA144A0443F1BC7
:102C20002D19B3685B1B5A1E93415B421D40F56032
:102C3000002F0DD033699D42E4D2013B5B1BB46889
:102C4000641BBC4200D93C009C42E0D91C00DEE77A
:102C50004846C0BCB946B046F8BD000010B5134C9C
:102C6000A8220021200000F086FD03232361636178
:102C70000F4AA2610F4BE3618023DB002362002334
:102C8000A3626362E36222660B4A62661022A26656
:102C90002367E3666367094A0F3204481178C15419
:102CA0000133013A102BF9D110BDC046C8010020F4
:102CB000943900088002002070020020A03900082A
:102CC000F8B503000F001600421C5400A418E400DD
:102CD000174AA4184000C018C0001218D56A012D68
:102CE00012D0022D1DD0002D02D000252800F8BDE5
:102CF0002000FFF749FF8642F8D832003900200053
:102D0000FFF74EFF3500F1E72000FFF73DFF3500EC
:102D1000864200D905002A0039002000FFF740FF55
:102D2000E4E732002000FFF762FF0500DEE7C0465F
:102D3000C8010020F8B504000D001600094B1B78EF
:102D4000532B0CD1EFF31087012181F3108832004F
:102D500029002000FFF7B4FF87F31088F8BDFFF7C4
:102D60007DFFEFE7C801002010B5FFF777FF10BD2A
:102D700010B504008268531C4068834205D820685F
:102D80008154A360E3680133E360A26863689A42F8
:102D900000D010BD21682069FFF7CCFFA3689842DE
:102DA00003D001235B42E360F3E70023A360F0E775
:102DB000F0B5DE4657464E464546E0B583B0804600
:102DC0000E0015001F000C9B994691422FD308005E
:102DD00001242900FDF798F901348542F9D9BB4651
:102DE000A74200D2A34601230D9A1A4001920D9AE0
:102DF00013421ED14B46002B1BD0202413009B07EF
:102E000006D53C00631E9C4164420F239C43303432
:102E1000D9450ED901235B429C46E144210040463E
:102E2000FFF7A6FF4346DB68002BF1DA34E001240C
:102E3000D5E74346DB68002B2EDB012401E0013F90
:102E40006C43012FFBD821003000FDF75DF985426E
:102E5000F6D91C4B9A4600E0040021003000FDF733
:102E600053F9070021003000FDF7D4F90E00534656
:102E7000D95D4046FFF77CFF4346DB68002B05DB4E
:102E800029002000FDF740F9AC42E5D2019B002B60
:102E900002D04B46002B06D103B0F0BCBB46B24675
:102EA000A946A046F0BDD945F6D901235B429C4610
:102EB000E14420214046FFF75BFF4346DB68002BDF
:102EC000F1DAE9E7803A0008F0B5DE4657464646B3
:102ED000C0B582B007008B4615009A460A9B9846FB
:102EE000CB17C8185840160090423CDB012429003B
:102EF000FDF794F90134B042F9DA5646A24500D202
:102F000026004346002B09D05B46002B02DB0B9BBF
:102F10005B0703D501235B429C46E0440B9B9B0768
:102F200002D55346002B05D00B9BDB0702D443464A
:102F3000002B1AD1FB68002B2EDB5B46002B22DB1B
:102F40000B9B5B072ED403230B9A1340022B2ED02E
:102F50000B9B01934346009353462A005946380081
:102F6000FFF726FF18E00124C7E74645E2D2012318
:102F70005B429C46E04420213800FFF7F9FEFB68E5
:102F8000002BF2DA08E05B429B462D213800FFF768
:102F9000EFFEFB68002BD6DA02B0E0BCBB46B246BF
:102FA000A846F0BD2B213800FFF7E2FEF1E75346BB
:102FB000002BCDD14346002BCAD046450BD201236E
:102FC0005B429C46E04430213800FFF7D1FEFB68AD
:102FD000002BF2DAE0E7FB68002BDDDBB8E700004E
:102FE000F0B5DE4657464E464546E0B5CBB00390B9
:102FF0000C00904605AB459380235B00469300236D
:1030000047934990489301339946914B9A4656E02D
:10301000002602201D39042208E0302B00D0FCE0FD
:103020000643013402E04B461E43013423782D2B26
:10303000F9D0F2D8232B05D02B2B00D0EDE016438E
:103040000134F3E70E430134F0E70025F8E0621C99
:1030500061780B00303B092B0DD80132BB00DB1926
:103060005B005B18303B1F0011780B00303B092BD5
:10307000F3D91400E8E014000027E5E001342378D8
:103080001A008A43682AF9D0252B6DD01A00463AD7
:10309000322A0FD8D2B2322A0CD893006D4AD358B4
:1030A0009F4643461B681A1D41460A60197845A889
:1030B000FFF75EFE0134489B002B00DA97E0217891
:1030C0000134002900D192E02529A1D045A8FFF7BD
:1030D0004FFEF0E743461B681A1D41460A60196817
:1030E000019600953B000A2245A8FFF7EDFEE1E7B7
:1030F00043461B681A1D41460A60196801960095EF
:103100003B000A2245A8FFF753FED3E743461B685E
:103110001A1D41460A601968019600953B0010226D
:1031200045A8FFF745FEC5E743461B681A1D414603
:103130000A601D68297801350029BBD045A8FFF732
:1031400017FE489B002BF5DAB4E743461B681A1DAF
:1031500041460A6019680023019308330093102246
:1031600045A8FFF725FEA5E7252145A8FFF700FEA6
:10317000A0E743461B680733072293431A0008322F
:1031800041460A6018685968FDF7A6FC834600218D
:10319000FDF742F9002825D15846FDF77DFCC317FD
:1031A000C1185940019600953B000A2245A8FFF737
:1031B0008BFE2E2145A8FFF7DBFD51465846FDF753
:1031C0001DFBFDF769FCC317C0185840FA218900A0
:1031D000FDF70AF90196009503230A2245A8FFF797
:1031E00073FE67E72D2145A8FFF7C2FDD4E7489D90
:1031F000002D04DD479C002C09D16419489448989F
:103200004BB0F0BCBB46B246A946A046F0BD22007A
:1032100005A90398FFF78EFDEFE722781300303BF6
:10322000092B00D911E700250134AB005B195B00C5
:103230009B18303B1D0022781300303B092BF3D93B
:1032400000272E2A00D102E72378042118E7C04680
:1032500000007A44B43900080FB400B583B004AB61
:1032600002CB019301AA0020FFF7BAFE03B008BC0D
:1032700004B0184710B5FFF777FD10BD70B50029F1
:1032800015D045180E4B01240E490CE05B08013A9D
:10329000002A05D01C42F9D05B084B409BB2F6E7F0
:1032A0000130854204D0027853400822F2E7044BF3
:1032B0005BBA9CB204482100FFF7CEFF200070BD2E
:1032C000FFFF000001A0FFFF903A000870B5040066
:1032D00012482100FFF7C0FF21681148FFF7BCFF2B
:1032E00061681048FFF7B8FF23680F4A1340802237
:1032F0009205934204D00D48FFF7AEFF012070BD48
:1033000065680B482900FFF7A7FF6420FEF7A8F8BF
:1033100072B6236883F30888A847EFE79C3A000851
:10332000AC3A0008C03A00080000FF2FE03A00085D
:10333000D03A0008F8B507000D00160072B6FEF787
:10334000FBF9002E0ED00B4BFC18A619ED1B0A4BF7
:103350009C4665442A5D21000020FEF725FA0134D1
:10336000B442F7D1FEF702FA62B60A20FEF778F807
:10337000F8BDC046000008080000F8F710B5094B7A
:10338000C318002A0DD0074CA44662441218091A2B
:10339000054884466144180001330078585493422C
:1033A000F9D110BD00000808FFFFF7F770B5050060
:1033B0000E0072B6FEF7C0F9002E12D000240020D5
:1033C0000B4B9C46654404E00434E4B22000B44254
:1033D00007D22818FEF7D4F90028F5D0013CE4B252
:1033E000F2E7FEF7C3F962B60A20FEF739F870BDBE
:1033F0000000080870B584B005000C000C22002104
:1034000001A800F0B8F900260096FEF7F3F801963F
:1034100002950394694601A8FEF70AFA041E03D038
:103420000124200004B070BDFEF714F9F9E7F0B5EF
:10343000C64600B506000F00150003231A002A40F7
:1034400090462B4205D001239846404680BCB846A2
:10345000F0BDFEF7CFF8002D0AD000243A593119FB
:103460000220FEF747F9002805D10434A542F5D81B
:10347000FEF7F0F8E9E701239846E6E7002A07D0CF
:1034800012180300091A1878C85401339342FAD16C
:103490007047000010B50A00034C044B01002000E7
:1034A000FFF790F810BDC04654010020FFFF000058
:1034B00010B582B00400A02000221021C005FEF744
:1034C000F9FA0120FDF7CCFF013C63425C41640046
:1034D00004346B46D81D04700121FFF7DBFF0400A4
:1034E000A02001221021C005FEF7E4FA631E9C41D2
:1034F000E0B202B010BD000030B583B004000D0092
:10350000A02000221021C005FEF7D4FA0120FDF70B
:10351000A7FF013C63425C416442302323400533F2
:103520006A46D01D03700121FFF7B4FF0124002873
:1035300008D0A02001221021C005FEF7BBFA200010
:1035400003B030BD0448054B01222900FFF754FAAF
:10355000431E9841C4B2ECE754010020FFFF000075
:1035600030B583B06B46DC1D012521000020FFF73C
:10357000C3FF23782B402370F7D103B030BD000088
:1035800070B582B00D00160001AC03232370030C4C
:103590006370030AA370E070FFF7E2FFA02000222F
:1035A0001021C005FEF786FA0120FDF759FF04211E
:1035B0002000FFF76FFF0124002808D0A02001227F
:1035C0001021C005FEF776FA200002B070BD054854
:1035D000054B32002900FFF70FFA431E9841C4B291
:1035E000ECE7C04654010020FFFF000070B582B038
:1035F0000D00160001AC02232370030C6370030A54
:10360000A370E070FFF7ACFF0120FFF751FFFFF759
:10361000A7FFA02000221021C005FEF74BFA0120D1
:10362000FDF71EFF04212000FFF734FF01240028CE
:103630000AD0A02001221021C005FEF73BFAFFF7B7
:103640008FFF200002B070BD31002800FFF722FF7D
:10365000431E9841C4B2ECE730B583B00023019318
:10366000D8336A4613715071FFF77AFF0120FFF7D4
:103670001FFFFFF775FFA025ED0500221021280090
:10368000FEF718FA0120FDF7EBFE042101A8FFF771
:1036900001FF0400012210212800FEF70BFAFFF7BA
:1036A0005FFF631E9C41E0B203B030BD30B583B014
:1036B00001AB214A12881A8000229A706B46DC1CEA
:1036C0009F232370FFF74CFFA02000221021C0058C
:1036D000FEF7F0F90120FDF7C3FE01212000FFF7FE
:1036E000D9FE00280AD0A02001221021C005FEF733
:1036F000E1F901241148FFF7AFFD19E01048114B23
:10370000032201A9FFF778F905000400631E9C411C
:10371000E4B2A02001221021C005FEF7CBF9002D54
:10372000E8D101A98B784A7809780748FFF794FD1A
:10373000200003B030BDC046FC370008003B000845
:1037400054010020FFFF0000EC3A000810B5020011
:1037500010210248FEF7AEF910BDC0460008005027
:1037600010B50120FFF7F2FF6420FDF779FE00207D
:10377000FFF79CFF10BD03008218934200D17047F1
:1037800019700133F9E7000070B500260C4C0D4D9F
:10379000641BA410A64209D1002600F023F80A4CAD
:1037A0000A4D641BA410A64205D170BDB300EB58AE
:1037B00098470136EEE7B300EB5898470136F2E739
:1037C000183B0008183B00081C3B0008183B000889
:1037D000002310B59A4200D110BDCC5CC454013313
:1037E000F8E70000F8B5C046F8BC08BC9E46704734
:0C37F000F8B5C046F8BC08BC9E46704707
:1037FC00000000007665723A20257825782578251A
:10380C00780D0A0073697A656F663A2025640D0A93
:10381C00000000007061636B6574733A2025640DC1
:10382C000A0000006C656E6774683A2025640D0A06
:10383C000000000063726331363A2025780D0A00CF
:10384C00424F4F5420494E4954204F4B0D0A000013
:10385C004D4F44455F53544152540D0A0000000033
:10386C00737461746520726561643A5B25785D0DD3
:10387C000A0000006576656E743D25780D0A00001F
:10388C006A756D705F6661696C0D0A005354455022
:10389C005F4241434B55500D0A000000775F626157
:1038AC00636B75705F636E742025640D0A000000F5
:1038BC00535445505F5245504C4143450D0A00004E
:1038CC0025782025640D0A00775F72756E5F636E34
:1038DC00742025640D0A0000535445505F4348453D
:1038EC00434B0D0A0000000074656D705F31363D6E
:1038FC0025780D0A0000000063726331365F737522
:10390C0063630D0A0000000063726331365F666109
:10391C00696C0D0A00000000535445505F4241434E
:10392C004B55505F434F50590D0A0000775F72653D
:10393C00636F7665725F636E742025640D0A0000F8
:10394C004241434B55505F6D6573736167652065EC
:10395C0072720D0A00000000486172644661756C59
:10396C00745F48616E646C65720D0A0000000000A3
:10397C0000000000010203040607080903040608FE
:10398C000C101820300000005465726D696E616C6B
:10399C00000000000000000000005454522052456A
:1039AC00474745530000000072310008B43000084E
:1039BC00B4300008B4300008B4300008B43000084B
:1039CC00B4300008B4300008B4300008B43000083B
:1039DC00B4300008B4300008B4300008B43000082B
:1039EC00B4300008B4300008B4300008B43000081B
:1039FC000C310008B4300008B4300008B4300008B2
:103A0C00B4300008B4300008B4300008B4300008FA
:103A1C00B4300008B4300008B4300008A2300008FC
:103A2C00D4300008B430000872310008B4300008FB
:103A3C00B4300008B4300008B4300008B4300008CA
:103A4C00B4300008B4300008B4300008B4300008BA
:103A5C004A310008B4300008B4300008283100089E
:103A6C00B4300008F0300008B4300008B43000085E
:103A7C000C31000830313233343536373839414265
:103A8C00434445466372633D25780D0A00000000EF
:103A9C00616464722070203D2025780D0A000000BE
:103AAC00616464722064617461203D2025780D0A84
:103ABC00000000004952512061646472203D2025B1
:103ACC00780D0A006A756D705F6F6B3D25780D0A75
:103ADC00000000006A756D705F6572720D0A00005F
:103AEC00726561645F69643D202578202578202506
:103AFC00780D0A00726561645F69643D20657272BD
:043B0C000D0A00009E
:083B1000F4C9FF7F0100000071
:043B1800E9000008B8
:043B1C00C1000008DC
:0C3B200000002000010000000400000074
:040000050800137567
:00000001FF
